:10000000020085120A3712005AD2AF7BFF7A0A79B2
:10001000551200F87F017E00120A20D3E5279400D4
:100020007480948040EE1527E52770E8D3E5269488
:100030000074809480401EE4F508E508C3952650BE
:100040001474002508F582E43400F583E0FF120AF9
:1000500046050880E5E4F52680BA750940750A046E
:10006000750E00750DC2750C01750B007510017BC6
:10007000007A0079097F0412084F7D017F0112097F
:100080007A53BAFB22787FE4F6D8FD758128020006
:01009000036C
:100093000209CDE518240CF8E60518227809300783
:1000A30002780CE475F0011208190206692000EBCE
:1000B3007F2ED2008018EF540F2490D43440D4FF05
:1000C30030040BEF24BFB41A0050032461FFE51979
:1000D30060021519051CE51C7002051B30070D781D
:1000E30009E475F001120819EF0207D1020A5074EE
:1000F30003D2078003E4C207F5188B098A0A890B28
:10010300E4F519F51BF51CE51960077F201200D1F2
:1001130080F5751AFFC201C200C202C203C205C242
:1001230006C20812009FFF700D3007057F00120002
:10013300E2AF1CAE1B22B4255FC2D5C20412009FDE
:10014300FF24D0B40A00501A75F00A781930D50587
:1001530008B6FF0106C6A426F620D5047002D20312
:1001630080D924CFB41A00EF5004C2E5D2040202AE
:10017300E2D20180C6D20080C0D20280BCD2D58038
:10018300BAD20580B47F201200D12002077401B5D2
:10019300190040F1120096FF1200D102010AD208A1
:1001A300D2068095120096FB120096FA120096F979
:1001B3004A4B700679B37A037BFF20022EE5196060
:1001C3002A7E008E8275830012068260060EEE651B
:1001D3001A70F0C2D5EBC0E0EAC0E0E9C0E0EE126D
:1001E3000329D0E0F9D0E0FAD0E0FB120669FF6002
:1001F300AAEBC0E0EAC0E0E9C0E01200D1D0E024FD
:1002030001F9D0E03400FAD0E0FBE51A0460DCD554
:100213001AD980877BFF7A037925D202809C7910D3
:1002230080027908C206C2088008D2D5790A800400
:10023300790AC2D5E51A047002F51AE4FAFDFEFF45
:10024300120096FC7B08200113120096FD7B1030F0
:10025300000A120096FE120096FF7B20EC3382D533
:1002630092D55013C3E43000069FFFE49EFEE420C2
:1002730001039DFDE49CFCE4CBF8C201EC700CCFC0
:10028300CECDCCE824F8F870F38017C3EF33FFEE3C
:1002930033FEED33FDEC33FCEB33FB994002FB0FF4
:1002A300D8E9EB300105F8D0E0C448B201C0E00A58
:1002B300EC4D4E4F78207B0070C2EAB51A0040BC6B
:1002C300C0E012032BD0F0D0E0200104C4C0E0C48E
:1002D300B201C0F01200BAD0F0D5F0EB02010A125D
:1002E300082901A75302215801784C0174420225C1
:1002F3004F022D44022D49018D4302335502174607
:1003030002174502174703D350017C2D01802E01AC
:10031300A32B01842301A12003BC2A013C48000034
:10032300019B3F3F3F00790AA2D520031430050902
:10033300B910020404B9080104A2D5200602500131
:10034300042002689202B519005034C0E07F2030C7
:1003530003197F30A20272067205500F120382C284
:1003630002C206C205C2087F30800F300503E9C010
:10037300E01200D1300503D0E0F9D0E0B519CC305C
:1003830005177F30B9100C1200D17F583004077F56
:10039300788003B908031200D13002057F2D0200D3
:1003A300D17F202008F87F2B2006F322920280CFF2
:1003B300286E756C6C2900D2011200963001F8C2C8
:1003C30001781930D50108F602013C2D50434958F4
:1003D3001200962403B405004001E49003CE931267
:1003E30000C2743A1200C2D203751904020221EF4B
:1003F300D394077480948040037FFF22120669FE22
:10040300D394037480948040037FFF22EF7044EE03
:10041300700B900001120682F452935294120669F3
:100423006401700B9000011206824293F4529412FD
:100433000669FE6402700A9000011206824293422A
:1004430094EE6403700D900001120682FEF4529341
:10045300EE4294EF64017046120669FE700B900041
:1004630001120682F452915292EE6401700B9000D5
:10047300011206824291F452921206696402700AD2
:10048300900001120682429142921206696403703F
:100493000D900001120682FEF45291EE4292EF6437
:1004A300027046120669FE700B900001120682F478
:1004B30052955296EE6401700B900001120682422F
:1004C30095F452961206696402700A9000011206AE
:1004D30082429542961206696403700D90000112E0
:1004E3000682FEF45295EE4296EF640370461206BE
:1004F30069FE700B900001120682F452B152B2EE03
:100503006401700B90000112068242B1F452B212E0
:1005130006696402700A90000112068242B142B277
:100523001206696403700D900001120682FEF452F4
:10053300B1EE42B2EF64047046120669FE700B908E
:100543000001120682F452B352B4EE6401700B90B0
:10055300000112068242B3F452B4120669640270B7
:100563000A90000112068242B342B4120669640380
:10057300700D900001120682FEF452B3EE42B4EF06
:1005830064057046120669FE700B90000112068224
:10059300F452C952CAEE6401700B90000112068234
:1005A30042C9F452CA1206696402700A9000011229
:1005B300068242C942CA1206696403700D900001A3
:1005C300120682FEF452C9EE42CAEF640670461266
:1005D3000669FE700B900001120682F452CB52CCD6
:1005E300EE6401700B90000112068242CBF452CCF0
:1005F3001206696402700A90000112068242CB421D
:10060300CC1206696403700D900001120682FEF499
:1006130052CBEE42CCEF64077049120669FF7E00AD
:10062300700B900001120682F452E152E2EF640172
:100633004E700B90000112068242E1F452E2120660
:10064300696402700A90000112068242E142E212DA
:1006530006696403700D900001120682FFF452E1F3
:10066300EF42E27F0022BB010689828A83E02250A7
:1006730002E722BBFE02E32289828A83E49322BB40
:10068300010CE58229F582E5833AF583E0225006E1
:10069300E92582F8E622BBFE06E92582F8E222E597
:1006A3008229F582E5833AF583E4932275F0087590
:1006B3008200EF2FFFEE33FECD33CDCC33CCC5829A
:1006C30033C5829BED9AEC99E58298400CF582EE56
:1006D3009BFEED9AFDEC99FC0FD5F0D6E4CEFBE43E
:1006E300CDFAE4CCF9A88222B800C1B90059BA0006
:1006F3002DEC8BF084CFCECDFCE5F0CBF97818EF61
:100703002FFFEE33FEED33FDEC33FCEB33FB10D761
:1007130003994004EB99FB0FD8E5E4F9FA22781822
:10072300EF2FFFEE33FEED33FDEC33FCC933C9107D
:10073300D7059BE99A4007EC9BFCE99AF90FD8E0AF
:10074300E4C9FAE4CCFB2275F010EF2FFFEE33FE81
:10075300ED33FDCC33CCC833C810D7079BEC9AE8F4
:1007630099400AED9BFDEC9AFCE899F80FD5F0DA75
:10077300E4CDFBE4CCFAE4C8F922EB9FF5F0EA9E62
:1007830042F0E99D42F0E89C45F022E8600FECC39B
:1007930013FCED13FDEE13FEEF13FFD8F122BB01A3
:1007A3000DE58229F582E5833AF5830207F05007C8
:1007B300E92582F80207E3BBFE07E92582F8020771
:1007C300FCE58229F582E5833AF583020809BB013A
:1007D3000689828A83F0225002F722BBFE01F322AC
:1007E300E6FB08E6F908E6FA08E6CBF822E0F8A308
:1007F300E0F9A3E0FAA3E0FB22E2FB08E2F908E256
:10080300FA08E2CBF822E493F8740193F9740293A3
:10081300FA740393FB22FAE6FB0808E6F925F0F6DF
:1008230018E6CA3AF622D083D082F8E493701274A1
:100833000193700DA3A393F8740193F5828883E465
:10084300737402936860EFA3A3A380DF8B128A13F0
:100853008914EF64046003020977752203F523F515
:1008630024F525F526F527F528FFEFC3942074809A
:100873009480500F74202FF582E43400F583E4F064
:100883000F80E7E4FFEFC3942074809480500F74CB
:10089300002FF582E43400F583E4F00F80E7AB1218
:1008A300AA13A914120669FF7E0064C06008EF64EE
:1008B300406003020960EF64C04E7005438480808A
:1008C3000353847F9000021207A17F007E607D5452
:1008D3007C001206EB8F188E178D168C15E4FFFE25
:1008E3007D01FCAB18AA17A916A815C312077D40F2
:1008F300037FFF22C3E49518F518E49517F51774E1
:10090300019516F516E49515F515AB12AA13A9145E
:1009130090000112068264027026538EEF5384BF47
:10092300538EF7438E04AF18AE17AD16AC15780887
:1009330012078E8FD68518D753AFFB438E108020B6
:10094300438440AF18AE17AD16AC15780812078E66
:100953008FD28518D353D10F43D1A080037FFF22B9
:10096300900007120682C454F0FFE58454EF4FF55C
:10097300847F00227FFF22EFD39401748094805000
:100983000CEFC454F0FFE5AF54EF4FF5AFEDFF7E2E
:1009930000D3940374809480502DEF700653EEFDC2
:1009A30053DFFDEF64014E700653EEFD43DF02EFAC
:1009B30064024E700643EE0253DFFDEF64034E7094
:1009C3000643EE0243DF027F0022C0E0C083C08201
:1009D300C0D075D000C007E584540160295384FE5C
:1009E300E5287022C3E52694207480948040037523
:1009F3002600AF26052674002FF582E43400F58324
:100A0300E585F0752705E584540260065384FD757A
:100A13002500D007D0D0D082D083D0E0327DA37C14
:100A230008ED1D70011C144C70F7EF1F70011E14AC
:100A33004E70EA22750A0CE4F509FB7A007909FF86
:100A43000203F28F85752501E52570FC22AE0702AE
:100A53000A46535443382055415254342054657345
:0F0A6300742050726F6772616D6D65210D0A000E
:00000001FF
